:0400000020EF10F0ED
:1000080000C01EF001C01DF002C01CF003C01BF0B0
:1000180004C01AF005C019F008C018F009C017F09C
:100028000AC016F00BC015F0E1CF27F0E2CF28F098
:10003800E9CF25F0EACF26F0F3CF23F0F4CF24F070
:10004800F5CF22F0F8CF1FF0F7CF20F0F6CF21F050
:10005800F2AA1DD0F2A41BD0010E4724006E000E98
:100068004820016E00C047F001C048F0000E006E45
:100078004850005C02E14750130808E2010E4D6E3B
:10008800000E4E6ED59EF29A476A486AF29489EC41
:100098000BF022C0F5FF1FC0F8FF20C0F7FF21C0FA
:1000A800F6FF23C0F3FF24C0F4FF1EC000F01DC0FC
:1000B80001F01CC002F01BC003F01AC004F019C004
:1000C80005F018C008F017C009F016C00AF015C0EE
:1000D8000BF025C0E9FF26C0EAFF27C0E1FF28C0D2
:0400E800E2FF110022
:1000EC000B6A0A6A096A00500402F4CF09F0F3CFD4
:1000FC0008F001500502F4CF0BF0F3CF0AF00050DA
:10010C000502F3500926F4500A22E86A0B2201502A
:10011C000402F3500926F4500A22E86A0B2208C0A4
:10012C0000F009C001F00AC002F00BC003F012008D
:10013C001E0E0F014D6F100E0001EB6F040EEC6FD5
:10014C00EBC0E1FFECC0E2FFE69EEBC0E1FFECC0D0
:10015C00E2FFE69C040EEB25E16E000EEC21E26E54
:10016C00E68C180E656F040E666F65C0E1FF66C005
:10017C00E2FFE69E65C0E1FF66C0E2FFE69C040E6E
:10018C006525E16E000E6621E26EE68C020EEB2513
:10019C00E16E000EEC21E26EDFC0E6FFE0C0E6FF90
:1001AC00010EEB25E16E000EEC21E26E400EE66EC8
:1001BC00EBC0E9FFECC0EAFFEECF00F0EBC0E1FFD3
:1001CC00ECC0E2FF400E0014E66EEBC0E9FFECC0A1
:1001DC00EAFFEECF00F0EBC0E1FFECC0E2FF880ECF
:1001EC000010E66EEBC0EDF0ECC0EEF0040EEB1977
:0801FC00006E00C0EBF01200E0
:100204000401286B296B4AD00001E48F0401288182
:1002140000016051010A02E10401288354D0000165
:10022400E48F51D00001E48F040124BF16D024C40C
:1002340003F00F0E031603C000F0000E016E00362B
:1002440000900136E90E0024E96E000E0120EA6EEA
:10025400EECF04F0EECF05F015D024C403F00F0E5A
:10026400031603C000F0000E016E00360090013644
:10027400630E0024E96E000E0120EA6EEECF04F056
:10028400EECF05F004C0E9FF05C0EAFFEECF01F0B0
:1002940001A403D00401010E286F15D020C401F07D
:1002A4001F0E01160150000AAFE020C401F01F0E1A
:1002B40001160150010AB3E020C401F01F0E01161B
:1002C4000150020AAFE00001E4AF07D0280EE16F4D
:0C02D400040EE26FE481020EE56F1200E0
:1002E00004012251010A13E120C401F01F0E01167E
:1002F0000150000A0CE10001E48F04012151030ABE
:1003000004E1010E0001606F02D00001606B040186
:100310002251000AD8A48DD020C401F01F0E01166E
:100320000150020AD8A485D024C401F00F0E011692
:100330000150000AD8B47DD00001E48F040124BF2D
:1003400016D024C403F00F0E031603C000F0000EF5
:10035000016E003600900136E90E0024E96E000EB1
:100360000120EA6EEECF04F0EECF05F015D024C4E4
:1003700003F00F0E031603C000F0000E016E0036EE
:1003800000900136630E0024E96E000E0120EA6E33
:10039000EECF04F0EECF05F02151030A07E104C0CF
:1003A000E1FF05C0E2FF840EE66E43D024C400F0F6
:1003B0000F0E00164C0E026E0F0E036E005002263A
:1003C000D8B0032A02C0E9FF03C0EAFFFE0EEE1414
:1003D000006EEECF01F0FF0E011602C0E1FF03C078
:1003E000E2FF00C0E6FF01C0E6FF24AF11D004C069
:1003F000E1FF05C0E2FFE66A040E0418006E00C0CB
:1004000004F004C0E1FF05C0E2FF400EE66E11D02B
:1004100004C0E1FF05C0E2FF880EE66E040E04187A
:10042000006E00C004F004C0E1FF05C0E2FFC80E8A
:04043000E66E120062
:1004340020C401F01F0E01160150010A01E094D0FE
:1004440004012451000A01E08FD02151060A42E13F
:1004540037D00001D951010A17E1B20E006E250E02
:10046400016E000E026E120E0026000E0122022200
:1004740000C0E1F001C0E2F002C0E3F0090EE56F54
:10048400000EE66FC00EE46F25D00001D951010AB9
:1004940012E1240E006E260E016E000E026E00C0E4
:1004A400E1F001C0E2F002C0E3F0210EE56F000EBE
:1004B400E66FC00EE46F0ED00001800EE46F0AD028
:1004C40004012351210AC5E02351220ADEE023510D
:1004D400230AF2E020C401F0600E0116050E006E3E
:1004E400005004E00132019EFF0FFBD70150010AC6
:1004F40001E03AD026D038D037D0D40E0001E16FD5
:10050400000EE26F010EE56F000EE66FC10EE46FA0
:100514002BD00001800EE46F23C4D4F025D0000159
:10052400D60EE16F000EE26F010EE56F000EE66F6E
:10053400810EE46F19D00001800EE46F22C4D6F05E
:1005440013D004012151010AD6E02151090AD4E053
:100554002151020AD2E021510A0ADBE02151030AA7
:0A056400DEE021510B0AE7E012006F
:10056E00000E0001E65D02E1080EE55D10E2E5C059
:10057E0003F0E6C004F0DE51000A03E1010EDE6F67
:10058E0005D0DE51010A02E1020EDE6F04D0080E24
:10059E00036E000E046E63C0E1FF64C0E2FFE692DC
:1005AE0063C0E1FF64C0E2FFE69063C0E9FF64C090
:1005BE00EAFFEECF00F063C0E1FF64C0E2FF04503B
:1005CE000010E66E010E6325E16E000E6421E26EF0
:1005DE0003C0E6FF0350E55D006E0450E659016E60
:1005EE0000C0E5F001C0E6F0280EE76F040EE86FDC
:1005FE00E4B12FD0035004102BE0E1C0F6FFE2C0AF
:10060E00F7FFE3C0F8FF0900F5CF00F0E7C0E1FF08
:10061E00E8C0E2FF00C0E6FFE74BE82B010EE12544
:10062E00006E000EE221016E000EE321026E00C08C
:10063E00E1F001C0E2F002C0E3F0010E035C006ED7
:10064E00000E0458016E00C003F001C004F0D2D7B2
:10065E0024D00350041021E0E1C0E9FFE2C0EAFF1C
:10066E00E7C0E1FFE8C0E2FFEECFE6FFE74BE82B85
:10067E00010EE125006E000EE221016E00C0E1F0D8
:10068E0001C0E2F0010E035C006E000E0458016E14
:0C069E0000C003F001C004F0DCD7120023
:1006AA0004012051800AD8A478D0C00E0001E46F5A
:1006BA0069D00001B40E006E260E016E000E026EA5
:1006CA0000C0E1F001C0E2F002C0E3F0120EE56FF3
:1006DA00000EE66F62D00001030E006E000E016E7E
:1006EA0022C404F0000E056EFCDCD00E0024E96E74
:1006FA00000E0120EA6EEECFE1F0EECFE2F0EECF8F
:10070A00E3F0020EE125F66E000EE221F76E000E0E
:10071A00E321F86E0900F5CF00F00900F5CF01F0EA
:10072A0000C0E5F001C0E6F038D004012251000112
:10073A00DC5D23E3030E006E000E016E22C404F09A
:10074A00000E056ECEDC4F0E0024E96E000E01206D
:10075A00EA6EEECFE1F0EECFE2F0EECFE3F0E1C0E9
:10076A00F6FFE2C0F7FFE3C0F8FF0900F5CF00F09B
:10077A0000C0E5F0000EE66F01D0E46B0ED0000178
:10078A00E46B0BD004012351010A93E02351020ABE
:0C079A00A2E02351030AC9E0F2D71200CC
:1007A6000001E48F0F014D6B0001D56B22C4D9F017
:1007B600D951000A03E1100EEF6F03D0200EEF6F40
:0407C600BADC120087
:1007CA00010E00016125E96E000E6221EA6EEECF8C
:1007DA0000F000C002F0000E6B5D02E102506A5D9B
:1007EA0003E26AC002F00AD002506A5D006E000E8F
:1007FA006B59016E00C06AF001C06BF0036A0250C7
:10080A00035C1CE2280EE96E040EEA6E0350E92628
:10081A00D8B0EA2AEECF00F067C0E1FF68C0E2FF75
:10082A0000C0E6FF010E6725006E000E6821016E0A
:10083A0000C067F001C068F0032AE1D7000E006E1D
:10084A006B51005C02E16A51000828E2010E5D2446
:10085A00E16E000E5E20E26E080EE66E020E5D2468
:10086A00E16E000E5E20E26E280EE66E040EE66E63
:10087A0061C0E9FF62C0EAFFEECF00F000BC07D01A
:10088A005DC0E1FF5EC0E2FFC80EE66E06D05DC045
:10089A00E1FF5EC0E2FF880EE66E19D0010E5D240C
:1008AA00E16E000E5E20E26E080EE66E020E5D2418
:1008BA00E16E000E5E20E26E200EE66E040EE66E1B
:1008CA005DC0E1FF5EC0E2FF840EE66E699F120022
:0A08DA000001DD5301E0A9DD12006A
:1008E40065980001E4BF49D069AF28D0020E5C6E60
:1008F400010E6325E16E000E6421E26EE66A63C0B8
:10090400E1FF64C0E2FFC80EE66E010E5D24E16EF5
:10091400000E5E20E26E080EE66E020E5D24E16EAD
:10092400000E5E20E26E280EE66E040EE66E5DC0DA
:10093400E1FF5EC0E2FFC80EE66E1ED0010E5D242C
:10094400E16E000E5E20E26E080EE66E020E5D247D
:10095400E16E000E5E20E26E200EE66E040EE66E80
:100964005DC0E1FF5EC0E2FF8C0EE66E63C0E1FF96
:1009740064C0E2FF840EE66E82D069BF80D00401B9
:1009840020AF55D00001E6510401275D04E10001C8
:10099400E5510401265D04E226C4E5F027C4E6F02F
:1009A400E4DD010E5C6E010E5D24E16E000E5E203E
:1009B400E26E080EE66E020E5D24E16E000E5E200D
:1009C400E26E200EE66E040EE66E5DC0E1FF5EC0D0
:1009D400E2FF800EE66E5F6A010E6125E16E000E95
:1009E4006221E26E080EE66E020E6125E16E000ED3
:1009F4006221E26E200EE66E040EE66E61C0E1FF37
:100A040062C0E2FF840EE66E010E5F6E020E632585
:100A1400E16E000E6421E26E280EE66E040EE66EB0
:100A240063C0E1FF64C0E2FFC80EE66E28D0000197
:100A3400020E5C6E010E6325E16E000E6421E26E0F
:100A4400E66A63C0E1FF64C0E2FFC80EE66E010E11
:100A54005D24E16E000E5E20E26E080EE66E020E6C
:100A64005D24E16E000E5E20E26E280EE66E040E3A
:100A7400E66E5DC0E1FF5EC0E2FFC80EE66E1200E6
:100A8400160E0F015F6F9F0E5D6F3B0E5C6F1200C1
:100A94005C6A63C0E1FF64C0E2FFE66A040E000121
:100AA4006319E16E64C0E2FF000EE21AE66A69AF00
:060AB40001D0699F120051
:100ABA0020C401F0600E0116050E006E005004E01D
:100ACA000132019EFF0FFBD70150000A01E060D0FE
:100ADA003CD00001E48F080EEF6F5AD0E1DD58D008
:100AEA005DDE56D00001D90EE16F000EE26FE4819F
:100AFA00010EE56FE48F4CD002EC01F049D070ECA6
:100B0A0001F046D0D50E006E000E016E040124518C
:100B1A000026D8B0012A00C0E1F001C0E2F00001CD
:100B2A00E481010EE56FE48F33D00001E48FD50E26
:100B3A00E16E000EE26E04012451E126D8B0E22AE9
:100B4A0022C4E6FF25D024D023D004012151050A6E
:100B5A00C0E02151060AC2E02151090AC1E021512F
:100B6A00080AC0E02151000AC7E02151010AC7E082
:100B7A002151030AC4E021510A0AC4E021510B0A97
:100B8A00D4E02151070ADFE021510C0ADDE0DCD76D
:020B9A00120047
:100B9C00B20E0001D06F250ED16F000ED26F440E35
:100BAC004F6E270E506E000E516E000E526E260EBA
:100BBC00536E000E546E840E556E250E566E000E3E
:040BCC00576E12004E
:100BD0005C50020A02E1F9DD1ED05CDF5F50000AC2
:100BE00019E1010E5D24E16E000E5E20E26E080E3A
:100BF000E66E020E5D24E16E000E5E20E26E200EB7
:100C0000E66E040EE66E5DC0E1FF5EC0E2FF8C0E94
:080C1000E66E01D05F6A1200DC
:100C180065920F015C9562A403D0FB0E6216FBD7A8
:020C28001200B8
:100C2A00040E00016319006E00C063F0EF51080A58
:100C3A000DE122C45EFF0F015E51000804E2100EAE
:100C4A000001EF6F03D00001040EEF6F5C50010A40
:100C5A003AE1020E6325E16E000E6421E26E280E6F
:100C6A00E66E040EE66E7EDCDE51020A07E163C020
:100C7A00E1FF64C0E2FF840EE66E24D0040E63191D
:100C8A00006E00C063F063C0E9FF64C0EAFFEECF04
:100C9A0000F000BC0CD0040E6319006E00C063F0B3
:100CAA0063C0E1FF64C0E2FFC80EE66E0BD0040E1B
:100CBA006319006E00C063F063C0E1FF64C0E2FF25
:0A0CCA00880EE66E01D0E1DE120094
:100CD40063C0E9FF64C0EAFFEECF00F000AE05D0C8
:100CE40063C0E1FF64C0E2FFE66A0001DE6B5C6A98
:0E0CF400E56BE66BE46BDFDEEEDDF2DD120099
:100D02004CDFED6BEE6BF06BF16B636A626AB9DE1E
:100D1200658C5E6B4D6B659C0001D76BD86B000ECA
:100D2200D85D02E1080ED75D17E2D7C000F0D8C047
:100D320001F0003600900136003600900136000EB8
:100D42000024E16E040E0120E26EE66AE66AE66ABB
:100D5200E66AD74BD82BE3D7160E0F014C6F62A66B
:100D620003D0F70E6216FBD70001E46B696B6A6B66
:100D72006B6B6598080E636F040E646FD96BEF6B33
:020D820012005D
:0C0D84000F015C85EF0E62166582120004
:040D9000A198120014
:100D94000F014CA119D061C0E9FF62C0EAFFEECF98
:100DA40001F00150800A0FE163C0E9FF64C0EAFF6B
:100DB400EECF01F00150840A06E161C0E1FF62C098
:0E0DC400E2FF8C0EE66E4C91DF0E62161200FE
:100DD2000001EF51000A0BE1656A0F015C6B51DE05
:100DE20065B602D06586FCD7010E0001EF6FEF51A8
:100DF200010A0AE165BA08D0626A0F015C6B5C8184
:100E02005C89020E0001EF6F62A406D00F015CA59F
:100E120003D0FB0E6216FFDE65A202D0B8DFDFD080
:100E220062A019D00F015CA116D06ADF040EEF6F29
:100E3200200E0401026F040E036F080E016F000EF4
:100E42000015006E00C000F48C0E0011006E00C090
:100E520000F4FE0E621662A806D00F015CA903D050
:100E620090DFEF0E621662AC05D00F015CAD02D0CE
:100E7200BF0E621662AA04D00F015CAB01D089DFFB
:100E820062A204D00F015CA301D0636A040E0001C8
:100E9200EF5D02E27CDFA3D00F015CA79FD00101CE
:100EA2000C6B040E0C5DD8B099D062A693D064CFBF
:100EB200D3F0F70E6216780E0001D315016E0150C1
:100EC200000AD8A486D0FD0ED315016E026AFF0E69
:100ED2000216000E021802E1000E01186CE17E0EED
:100EE200D315016E01C003F00332039E03C000F06C
:100EF200000E016E00360090013600360090013679
:100F0200000E0024026E040E0120036E02C061F086
:100F120003C062F002C05DF003C05EF0040E5D1813
:100F2200006E00C05DF002C0E9FF03C0EAFFEECF31
:100F320000F000C001F03C0E01160132019E0132A8
:100F4200019E01500D0A35E1020E6125E96E000E87
:100F52006221EA6EEECF01F0EECF02F00250040AF7
:100F620002E1280E011823E1020E6125E16E000E56
:100F72006221E26E200EE66E040EE66E01010B6B3C
:100F8200080E0B5D14E2200EE16E040EE26E0B51B0
:100F9200E126D8B0E22A280EE96E040EEA6E0B5161
:100FA200E926D8B0EA2AEECFE6FF0B2BE9D791DE8D
:100FB20001D00DDE0DD0FD0ED315016E026AFF0EBB
:100FC2000216000E021802E1040E011801E12CDEE5
:100FD20000D001D003D001010C2B63D7D8DE120060
:100FE2000BC1C9FF016A0150000A05E1000EC7B03A
:0C0FF200010E016EF8D7C9CF01F012000B
:100FFE0001010C51000A12E00BC100F0000E016E4F
:10100E00003600900136630E0024E96E000E0120BA
:10101E00EA6EEECF04F0EECF05F011D00BC100F06A
:10102E00000E016E003600900136E90E0024E96EC6
:10103E00000E0120EA6EEECF04F0EECF05F0020EA8
:10104E000424E16E000E0520E26E0DC1E6FF0EC116
:10105E00E6FF010E0424E16E000E0520E26E0FC1C4
:10106E00E6FF04C0E9FF05C0EAFFEECF00F004C0C2
:10107E00E1FF05C0E2FF400E0014E66E04C0E9FF7A
:10108E0005C0EAFFEECF00F004C0E1FF05C0E2FFAD
:10109E00880E0010E66E0C51000A1BE00BC100F02A
:1010AE00000E016E003600900136630E0024026EB3
:1010BE00000E0120036E02C0E9FF03C0EAFF040E1A
:1010CE00EE18006E02C0E1FF03C0E2FF00C0E6FFB3
:1010DE001AD00BC100F0000E016E003600900136E2
:1010EE00E90E0024026E000E0120036E02C0E9FF1D
:1010FE0003C0EAFF040EEE18006E02C0E1FF03C04B
:10110E00E2FF00C0E6FF04C000F005C001F01200CF
:10111E00000E01010C1902E1000E0B1902E1016A29
:10112E000AD00BC1E9FF0CC1EAFFEECF00F0000EB2
:0C113E0000BE010E016E01C000F01200A6
:0E114A008C928F8000C10BF147DF8C82120067
:10115800B40E006E260E016E000E026E0E0E0024F6
:10116800F66E000E0120F76E000E0220F86E0900E0
:10117800F5CF03F003C004F00F0E0024F66E000E46
:101188000120F76E000E0220F86E0900F5CF01F07D
:101198000150035C12E2B40E006E260E016E000EC2
:1011A800026E0F0E0024F66E000E0120F76E000E80
:1011B8000220F86E0900F5CF04F0B40E006E260E7A
:1011C800016E000E026E100E0024F66E000E012055
:1011D800F76E000E0220F86E0900F5CF01F00150FD
:1011E800045C12E2B40E006E260E016E000E026E52
:1011F800100E0024F66E000E0120F76E000E02207D
:0E120800F86E0900F5CF04F004C000F01200EB
:101216000101006B086B096B020E0525F66E000EC8
:101226000621F76E000E0721F86E0900F5CF05F0CE
:10123600030E0525F66E000E0621F76E000E072139
:10124600F86E0900F5CF00F000C003F0000E046E42
:1012560003C001F0006A05500024066E000E01204E
:10126600076E05C108F006C109F007C10AF0010EB4
:101276000824F66E000E0920F76E000E0A20F86E9E
:101286000900F5CF01F00150020A1BE1060E082401
:10129600F66E000E0920F76E000E0A20F86E0900A1
:1012A600F5CF01F00150005D0CE2060E0824F66E43
:1012B600000E0920F76E000E0A20F86E0900F5CF21
:1012C60000F1010E0824F66E000E0920F76E000EDE
:1012D6000A20F86E0900F5CF01F00150040A1BE15F
:1012E600080E0824F66E000E0920F76E000E0A207E
:1012F600F86E0900F5CF01F00150005D0CE2080E12
:101306000824F66E000E0920F76E000E0A20F86E0D
:101316000900F5CF00F108C0F6FF09C0F7FF0AC0C3
:10132600F8FF0900F5CF00F000500825016E000E09
:101336000921026E01C008F102C009F10750025CE2
:1013460002E10650015C01E30FD008C0F6FF09C0B8
:10135600F7FF0AC0F8FF0900F5CF00F00050082695
:0E136600000E09220A2283D700C100F01200F7
:0A137400D08EA288A088F28E12002D
:10137E00200E0001EF5D03E365B201D002D0006ADA
:10138E0049D0F0C00BF1F1C00CF1C2DE005241E1C8
:10139E0008C10BF1010E0C6F05C10DF106C10EF166
:1013AE0007C10FF125DE00C0F0F001C0F1F0000121
:1013BE00F26BF36BF46BF56BF0C00BF1F1C00CF14B
:1013CE00A7DE00520FE0010E016E0150000A01E18E
:1013DE00F9DC0001F251F311F411F51102E0006A8B
:1013EE0019D0EAD70001F0C009F1F1C00AF1000EE0
:1013FE00F11902E1000EF0190AE0010E01010925B2
:10140E00E96E000E0A21EA6EEECF00F003D0006AFC
:06141E0001D0006A12007B
:101424008C928F9005C10BF1DADD8C828C928F80C7
:0A14340006C10BF1D4DD8C8212001A
:10143E00340E0101056F01C106F1EDDF350E01011C
:10144E00056F02C106F1E7DF360E0101056F03C11C
:10145E0006F1E1DF370E0101056F04C106F1DBDF96
:02146E0012006A
:0E147000570E0D6E0D2EFED70000000012006C
:10147E008C928F90080E01010B6FACDD8C821200E6
:10148E0064DE00C0FDF0B20E0101056F250E066F81
:10149E00000E076FB9DE00C0FEF00001FD51005CCA
:0E14AE0003E2FDC000F002D0FEC000F012000C
:1014BC00086A096A100E0C6E01340836093604509D
:1014CC00085E0550D8A0053C095ED8B007D0045082
:1014DC0008260550D8B0053C0926D89000360136B0
:0614EC000C2EEAD71200ED
:1014F2000001EF51000A0DE1656A0F015C6B42ECDD
:1015020005F037DF65B602D06586FCD7010E000113
:04151200EF6F120065
:10151600FDC005F1FEC006F1FFC007F1010E010195
:06152600086F2ADF12002D
:0E152C00FDC000F10CDEFEC000F109DE120071
:10153A000001FF6B200EEF5D03E365B201D002D01C
:10154A00006A2FD0EDC00BF1EEC00CF1E3DD0052C2
:10155A0027E1EDC0FDF0EEC0FEF0000E0001EE192D
:10156A0002E1000EED190AE0010EFD25E96E000EFA
:10157A00FE21EA6EEECF00F000C0FFF004C10BF1CD
:10158A0001010C6B01C10DF102C10EF103C10FF192
:10159A0031DD00C0EDF001C0EEF0FFC000F001D077
:0415AA00006A1200C1
:1015AE00F6C004F0F7C005F004C002F005C003F069
:1015BE00044A052AF8C000F0F9C001F00001F84B0A
:1015CE00F92B00C0E9FF01C0EAFF02C0E1FF03C032
:1015DE00E2FFEECFE6FF02C0E9FF03C0EAFFEE52E4
:0E15EE0001E0E2D7F6C000F0F7C001F01200F5
:1015FC000900F5CFE6FF0006FBE10106F9E1120058
:10160C000D0E0501406F0A0E416F426B400E00013A
:10161C00FD6F050EFE6F400EFF6F77DF005201E18C
:04162C00F5D71200DC
:10163000F8C0F6FFF9C0F7FFFAC0F8FF0900F5CFD0
:1016400000F0005218E0F8C0F6FFF9C0F7FFFAC04A
:10165000F8FF0900F5CF00F0F6C0E1FFF7C0E2FFA8
:1016600000C0E6FF0001F64BF72B010EF827000E35
:10167000F923FA23DDD7F6C0E1FFF7C0E2FFE66AFF
:02168000120056
:10168200FE0EC16EFF0EC26EFF0E926EFF0E946EC4
:10169200FF0E986E929295909592989089928C9066
:1016A2008C928F90958E9986959896988C988D9815
:0216B200120024
:1016B4008C883D0E0B6EE10E0C6E3F0E0D6E0D2EE2
:1016C400FED70C2EFCD70B2EFAD7000000008C9806
:1016D4003D0E0B6EE10E0C6E3F0E0D6E0D2EFED701
:1016E4000C2EFCD70B2EFAD7000000008C883D0E80
:1016F4000B6EE10E0C6E3F0E0D6E0D2EFED70C2EF2
:0E170400FCD70B2EFAD7000000008C981200C4
:101712000001EF51010A09E165BA07D0626A0F01BF
:101722005C815C89020E0001EF6F62A407D00F0199
:101732005CA504D0FB0E62160CEC06F065A203D089
:10174200C8EC06F0E7D062A01AD00F015CA117D056
:1017520081EC06F0040EEF6F200E0401026F040EFE
:10176200036F080E016F000E0015006E00C000F43A
:101772008C0E0011006E00C000F4FE0E621662A80C
:1017820007D00F015CA904D0C2EC06F0EF0E62167E
:1017920062AC05D00F015CAD02D0BF0E621662AA28
:1017A20005D00F015CAB02D0CAEC06F062A204D0F5
:1017B2000F015CA301D0636A040E0001EF5D03E236
:1017C200C8EC06F0A7D00F015CA7A2D00101116BF3
:1017D200040E115DD8B09CD062A696D064CFD3F02F
:1017E200F70E6216780E0001D315016E0150000A41
:1017F200D8A489D0FD0ED315016E026AFF0E02161F
:10180200000E021802E1000E01186EE17E0ED315E1
:10181200016E01C003F00332039E03C000F0000E0C
:10182200016E003600900136003600900136000E3F
:101832000024026E040E0120036E02C061F003C098
:1018420062F002C05DF003C05EF0040E5D18006E2F
:1018520000C05DF002C0E9FF03C0EAFFEECF00F076
:1018620000C001F03C0E01160132019E0132019EC0
:1018720001500D0A36E1020E6125E96E000E622169
:10188200EA6EEECF01F0EECF02F00250040A02E15E
:10189200280E011823E1020E6125E16E000E62217D
:1018A200E26E200EE66E040EE66E0101106B080E6B
:1018B200105D14E2200EE16E040EE26E1051E1267C
:1018C200D8B0E22A280EE96E040EEA6E1051E9261B
:1018D200D8B0EA2AEECFE6FF102BE9D76AEC06F081
:1018E20002D0E8EC05F00ED0FD0ED315016E026AAF
:1018F200FF0E0216000E021802E1040E011802E1A8
:1019020015EC06F000D001D003D00101112B60D7F5
:06191200C8EC06F0120013
:101918008C988D981F0E0B6E710E0C6E1E0E0D6E30
:101928000D2EFED70C2EFCD70B2EFAD700008C8874
:101938001F0E0B6E710E0C6E1E0E0D6E0D2EFED749
:101948000C2EFCD70B2EFAD700008C988D881F0E12
:101958000B6E710E0C6E1E0E0D6E0D2EFED70C2E1C
:10196800FCD70B2EFAD700008C888D981F0E0B6EB3
:10197800710E0C6E1E0E0D6E0D2EFED70C2EFCD7A2
:0C1988000B2EFAD700008C988D981200EE
:101994007CDD00C0DCF0010EDD6FF6C0DFF0F7C0C7
:1019A400E0F0F8C0DAF0F9C0DBF081EC06F0010EEB
:0C19B400016E0150010A01E19ADD1200F1
:1019C000C29EC29CC29AC298C296C294C280010EA4
:1019D000C26EC18EC19CC18AC188C196C182C184B8
:0419E000C1901200A0
:1019E4008C909C0E0C6ED70E0D6E0D2EFED70C2E09
:1019F400FCD78C809C0E0C6ED70E0D6E0D2EFED770
:101A04000C2EFCD7010E0101056F066B09DD140EC7
:101A14000101056F010E066F03DD4E0E0C6EEB0E19
:101A24000D6E0D2EFED70C2EFCD7140E0101056F82
:101A3400066BF6DC4E0E0C6EEB0E0D6E0D2EFED705
:101A44000C2EFCD7020E0101056F066BE9DC0F0EAC
:101A54000101056F066BE4DC1A0E0101056F030E2C
:101A6400066FDEDC300E0101056F066BD9DC310E2A
:101A74000101056F5F0E066FD3DC320E0101056FA5
:101A8400066BCEDC330E0101056F5F0E066FC8DCFA
:101A9400E00E0101056F066BC3DCE10E0101056F69
:101AA400066BBEDCE50E0101056F800E066FB8DC27
:101AB4000D0E0101056F066BB3DC1D0E0101056FF0
:101AC400066BAEDC090E0101056F066BA9DC130E73
:101AD4000101056F066BA4DC400E0101056F6E0E5B
:101AE400066F9EDC410E0101056F4F0E066F98DCF8
:101AF400420E0101056F770E066F92DC480E01015C
:101B0400056F066B8DDC180E0101056F010E066F63
:101B140087DC160E0101056F066B82DC3A0E0101AB
:101B2400056F020E066F7CDC3B0E0101056F020E91
:101B3400066F76DC3C0E0101056F020E066F70DC49
:101B44003D0E0101056F140E066F6ADC3E0E0101A5
:101B5400056F500E066F64DC3F0E0101056F190E10
:101B6400066F5EDC170E0101056F066B59DC490E2A
:101B74000101056F040E066F53DC380E0101056F79
:101B8400066B4EDC390E0101056F066B49DC020E53
:0C1B94000101056F010E066F43DC12001A
:101BA000D596D584D592D590D59AD59C6D0ED76E05
:101BB000840ED66EF294476A486A4D6A4E6AF18482
:061BC000F28AD58E12002E
:101BC600FAC000F00001FA07005228E0F6C0E9FF6B
:101BD600F7C0EAFFEE50000A0CE0F6C0E9FFF7C0D6
:101BE600EAFFF8C0D9FFF9C0DAFFEE50DE1801E1CE
:101BF6000FD0F6C0E9FFF7C0EAFFF8C0D9FFF9C079
:101C0600DAFFDE50EE5C006E016A000E015A08D063
:101C16000001F64BF72BF84BF92BD2D7006A016A75
:021C26001200AA
:101C2800FF0E586EFF0E596EFF0E5A6EFF0E5B6E5A
:101C3800E20E496E0F0E4A6E0B0E4B6E010E4C6E85
:101C4800949A94969488C66A400EC76EC68A120003
:101C5800C26A070EC16EC18EF6C000F00036009051
:101C6800003600900050C212C28038EC0AF0C282DE
:101C7800C2A201D0FDD7C4CF01F0006AC350001240
:081C8800000E0112C2901200CF
:101C90000001FA6B050EFA5D0AE2FA51F825E16ED1
:101CA000000EF921E26E200EE66EFA2BF3D7FA5100
:101CB000F825E16E000EF921E26EE66AFA07FA51A4
:101CC000F825FB6F000EF921FC6F0A0E046E000E62
:101CD000056EF6C000F0F7C001F05EEC0AF008C037
:101CE00000F009C001F0300E0026FBC0E1FFFCC08F
:101CF000E2FF00C0E6FF0A0E046E000E056EF6C09D
:101D000000F0F7C001F05EEC0AF000C0F6F001C090
:101D1000F7F0000E011802E1000E001801E102D0F8
:061D2000FA07CDD7120006
:101D26001D0E0101056F020E066F12EC0AF001018D
:101D3600016B5F0E026F036B5F0E046F1FEC0AF000
:101D46003FEC0AF00001F66BF76B240EF75D02E13B
:101D5600000EF65D0AE2FF0EFD6FFF0EFE6F96ECBB
:101D66000AF00001F64BF72BF0D7050E0101016FC3
:101D76005A0E026F050E036F5A0E046F1FEC0AF01F
:101D86003FEC0AF00001F66BF76B1F0EF75D02E100
:101D9600A40EF65D0AE20C0EFD6FC00EFE6F96EC09
:101DA6000AF00001F64BF72BF0D73D0E0B6EE10E55
:101DB6000C6E3F0E0D6E0D2EFED70C2EFCD70B2E85
:101DC600FAD7000000000A0E0101016F550E026FDE
:101DD6000A0E036F550E046F1FEC0AF03FEC0AF073
:101DE6000001F66BF76B1C0EF75D02E1390EF65D2E
:101DF60009E2FF0EFD6FFE6B96EC0AF00001F64B52
:101E0600F72BF1D73D0E0B6EE10E0C6E3F0E0D6EED
:101E16000D2EFED70C2EFCD70B2EFAD70000000095
:101E26000F0E0101016F500E026F0F0E036F500E61
:101E3600046F1FEC0AF03FEC0AF00001F66BF76B3B
:101E4600190EF75D02E1000EF65D09E2800EFD6FE8
:101E5600FE6B96EC0AF00001F64BF72BF1D7140E49
:101E66000101016F4B0E026F140E036F4B0E046FD0
:101E76001FEC0AF03FEC0AF00001F66BF76B150E4B
:101E8600F75D02E1F90EF65D09E2F80EFD6FFE6BF5
:101E960096EC0AF00001F64BF72BF1D73D0E0B6ED0
:101EA600E10E0C6E3F0E0D6E0D2EFED70C2EFCD7DE
:101EB6000B2EFAD700000000190E0101016F460E25
:101EC600026F190E036F460E046F1FEC0AF03FEC0B
:101ED6000AF00001F66BF76B130EF75D02E1240EB4
:101EE600F65D09E2FD6BFF0EFE6F96EC0AF000014F
:101EF600F64BF72BF1D71E0E0101016F410E026F53
:101F06001E0E036F410E046F1FEC0AF03FEC0AF041
:101F16000001F66BF76B100EF75D02E1810EF65DC0
:101F26000AE2800EFD6FFF0EFE6F96EC0AF00001CE
:101F3600F64BF72BF0D7020E0A6E310E0B6E620EC1
:101F46000C6E450E0D6E0D2EFED70C2EFCD70B2EED
:081F5600FAD70A2EF8D7120099
:101F5E008D881F0E0B6E710E0C6E1E0E0D6E0D2EDD
:101F6E00FED70C2EFCD70B2EFAD700008D981F0E25
:101F7E000B6E710E0C6E1E0E0D6E0D2EFED70C2EF0
:101F8E00FCD70B2EFAD700008D881F0E0B6E710E2C
:101F9E000C6E1E0E0D6E0D2EFED70C2EFCD70B2EBC
:101FAE00FAD700008D981F0E0B6E710E0C6E1E0E62
:101FBE000D6E0D2EFED70C2EFCD70B2EFAD7000071
:101FCE008D881F0E0B6E710E0C6E1E0E0D6E0D2E6D
:101FDE00FED70C2EFCD70B2EFAD700008D981200D0
:101FEE00F6C002F0F7C003F002C000F003C001F02B
:101FFE00024A032A00C0E9FF01C0EAFFEE5201E0E7
:10200E00F3D70001F651025C006EF7510358016ED2
:0A201E00010E005E000E015A1200D0
:10202800DFC001F1E0C002F1400E0101036F010EB3
:08203800046F9DEC0AF0120098
:10204000A4EC13F041EC0BF07A0E0B6EC10E0C6E8B
:10205000810E0D6E0D2EFED70C2EFCD70B2EFAD74F
:10206000000000000001766BB66B760E746F000EF8
:10207000756F52DC000EF66F050EF76F400EF86FAD
:10208000050EF96F87DC06EC0BF07A0E0B6EC10EB5
:102090000C6E810E0D6E0D2EFED70C2EFCD70B2E66
:1020A000FAD7000000005AEC0BF0400E0001F66F6A
:1020B000050EF76F040EF86F270EF96F000EFA6F1A
:1020C00018EC0BF0400E0001FD6F050EFE6F400E88
:1020D000FF6F8BEC0AF0005201E1F4D706EC0BF035
:1020E000400E0001F66F050EF76F9D0EF86F260E7D
:1020F000F96F000EFA6F18EC0BF0400E0001FD6F47
:10210000050EFE6F400EFF6F8BEC0AF0005201E1EE
:10211000F4D706EC0BF0400E0001F66F050EF76FDA
:10212000310EF86F000EF96FD7EC0AF00001400E87
:10213000FD6F050EFE6F400EFF6F8BEC0AF0005234
:1021400001E1F4D7400E0001F66F050EF76F510E56
:10215000F86F000EF96FD7EC0AF00001400EFD6F2A
:10216000050EFE6F400EFF6F8BEC0AF0005201E18E
:10217000F4D7020E0A6E310E0B6E620E0C6E450E17
:102180000D6E0D2EFED70C2EFCD70B2EFAD70A2E75
:10219000F8D7E5DE49DD0D0E0B6E2D0E0C6ED70E59
:1021A0000D6E0D2EFED70C2EFCD70B2EFAD700008D
:1021B000000018DCB8DD04DC400EF66F050EF76F8A
:1021C000D60EF86F260EF96F000EFA6F18EC0BF0B2
:1021D000400E0001FD6F050EFE6F400EFF6F8BEC91
:1021E0000AF0005201E1F4D79D9AA39AF28CF28E84
:1021F000476A486AD5DC0001706B716B000E715D37
:1022000002E1080E705D25E2D20E0101056F70C07B
:1022100006F112EC0AF0D00E0101056F880E066F70
:1022200012EC0AF01F0E0B6E710E0C6E1E0E0D6E70
:102230000D2EFED70C2EFCD70B2EFAD70000D00E99
:102240000101056F066B12EC0AF00001704B712B57
:10225000D5D7A6DCE9DE005207E1000E4E1802E1F8
:10226000000E4D1801E1F6D7000E4E1802E1010EE6
:102270004D1802E195DCF7D0000E0001F66F050E57
:10228000F76FB5DE00C072F001C073F074C0F6F0F5
:1022900075C0F7F0000EF86F050EF96FD7EC0AF075
:1022A000400EF66F050EF76FE60EF86F260EF96F0B
:1022B000000EFA6F18EC0BF0400E0001FD6F050EDA
:1022C000FE6F400EFF6F8BEC0AF0005201E1F4D775
:1022D000400E0001F66F050EF76F74C0F8F075C080
:1022E000F9F0D7EC0AF00001400EFD6F050EFE6F0D
:1022F000400EFF6F8BEC0AF0005201E1F4D706ECC0
:102300000BF0000E0001F66F050EF76F290EF86F47
:10231000000EF96F060EFA6F56DC000E011802E18E
:10232000000E00181AE18C88400E0001F66F050EB1
:10233000F76F2E0EF86F270EF96F000EFA6F18EC7C
:102340000BF0400E0001FD6F050EFE6F400EFF6F9B
:102350008BEC0AF0005201E1F4D7000E0001F66F99
:10236000050EF76F380EF86F000EF96F070EFA6F53
:102370002ADC000E011802E1000E00181AE18C9808
:10238000400E0001F66F050EF76FF50EF86F260E82
:10239000F96F000EFA6F18EC0BF0400E0001FD6FA4
:1023A000050EFE6F400EFF6F8BEC0AF0005201E14C
:1023B000F4D7000E0001F66F050EF76F400EF86FB0
:1023C000000EF96F060EFA6FE3EC0DF0000E011827
:1023D00002E1000E00181AE18D88400E0001F66F30
:1023E000050EF76F390EF86F270EF96F000EFA6FB2
:1023F00018EC0BF0400E0001FD6F050EFE6F400E55
:10240000FF6F8BEC0AF0005201E1F4D7000E0001DF
:10241000F66F050EF76F300EF86F000EF96F070EAE
:10242000FA6FE3EC0DF0000E011802E1000E001847
:102430001AE18D98400E0001F66F050EF76F130E2E
:10244000F86F270EF96F000EFA6F18EC0BF0400EC4
:102450000001FD6F050EFE6F400EFF6F8BEC0AF062
:10246000005201E1F4D70001F66B2CEC0EF000C035
:10247000CEF001C0CFF000C0F6F001C0F7F0B60E0C
:102480000001F86F000EF96F03DC400EF66F050EC9
:10249000F76F220EF86F270EF96F000EFA6F18EC27
:1024A0000BF0B60E0001F66F000EF76FA0DD00C056
:1024B00072F001C073F0B60E0024E16E000E012030
:1024C000E26E0D0EE66EB60E7225006E000E7321E2
:1024D000016E010E0024E16E000E0120E26E0A0E74
:1024E000E66EB60E7225006E000E7321016E020EAE
:1024F0000024E16E000E0120E26EE66A470EF66FE0
:10250000050EF76FB60EF86F000EF96FD7EC0AF0F4
:102510000001400EFD6F050EFE6F400EFF6F8BEC4D
:102520000AF0005201E1F4D77A0E0B6EC10E0C6E68
:10253000810E0D6E0D2EFED70C2EFCD70B2EFAD76A
:082540000000000058D6FFD78F
:1027480010EE29F01E0E006E010E016E650EF66E7B
:0E275800260EF76E000EF86EFEEC0AF0120070
:1025480031384638374A353020436C69636B6572D9
:10255800323A2054657374204F4C4544204320532D
:1025680045505331313441203936783936203635A3
:0C2578004B20636F6C6F72730D0A200023
:102584002A03500049004300310038004600380057
:1025940037004A0035003000200043006C00690019
:0E25A40063006B006500720032000000000052
:1025B200090229000101008032090400000203001F
:1025C20000000921010100012221000705810340C9
:0925D200000107050103400001AE
:1025DB00417474656E746520496E6974206C696111
:1025EB0069736F6E20484944205465726D696E6142
:0525FB006C200D0A0038
:102600002403530061006200650072002000450051
:102610006C0065006300740072006F006E0069005A
:0426200063007300E0
:102624000600FF0901A10119012940150026FF0038
:102634007508954081021901294075089540910259
:01264400C0D5
:1026450050726F6A65743A204F6C65645F435F3101
:10265500384638374A35302E6D637070690D0A007B
:072665004C44315F4F4E00B1
:08266C004C44325F4F4646006A
:082674004C44315F4F46460063
:07267C004C44325F4F4E0099
:10268300513D384D485A207820504C4C203D3E2037
:0A26930034384D487A20200D0A006B
:10269D004F4C454420737572206D696B726F427596
:0726AD00732023320D0A0027
:1026B40012010002000000083412010001000102AE
:0226C400000113
:1026C6002E2E2E2E2E2E2E2E2E2E2E2E200D0A00A5
:1026D600496E742041444320636830200D0A20006F
:0F26E600526563657074696F6E2064653A2000F9
:0F26F50053687574646F776E204C44310D0A0082
:0F27040033312D30372D3230313520610D0A0041
:0F27130053687574646F776E204C44320D0A0062
:0C272200454130203D202E2E2E2E2000A0
:0B272E0046697265204C44310D0A0022
:0B27390046697265204C44320D0A0016
:04274400040309047D
:020000040001F9
:06FFF800ACF7C4FFF8FFA6
:00000001FF
